
 MCIOLE16

 Start     Length     Name                   Class
 0001:0000 011A2H     _TEXT                  CODE
 0002:0000 00048H     _DATA                  DATA
 0002:0048 00000H     CONST                  CONST
 0002:0048 00000H     _BSS                   BSS
 0002:0050 00140H     c_common               BSS

 Origin   Group
 0002:0   DGROUP

 Address   Export                  Alias

 0001:0678 DllCreate               DllCreate
 0001:0558 DllCreateFromClip       DllCreateFromClip
 0001:06DA DllCreateFromFile       DllCreateFromFile
 0001:0616 DllCreateFromTemplate   DllCreateFromTemplate
 0001:05BA DllCreateLinkFromClip   DllCreateLinkFromClip
 0001:0742 DllCreateLinkFromFile   DllCreateLinkFromFile
 0001:04F0 DllLoadFromStream       DllLoadFromStream
 0001:03DC OleQueryObjPos          OleQueryObjPos
 0001:0070 WEP                     WEP

  Address         Publics by Name

 0000:0000  Imp  CLIENTTOSCREEN       (USER.28)
 0000:0000  Imp  CREATEBITMAP         (GDI.48)
 0000:0000  Imp  CREATECOMPATIBLEDC   (GDI.52)
 0000:0000  Imp  DEFCREATE            (OLECLI.DEFCREATE)
 0000:0000  Imp  DEFCREATEFROMCLIP    (OLECLI.DEFCREATEFROMCLIP)
 0000:0000  Imp  DEFCREATEFROMFILE    (OLECLI.DEFCREATEFROMFILE)
 0000:0000  Imp  DEFCREATEFROMTEMPLATE (OLECLI.DEFCREATEFROMTEMPLATE)
 0000:0000  Imp  DEFCREATELINKFROMCLIP (OLECLI.DEFCREATELINKFROMCLIP)
 0000:0000  Imp  DEFCREATELINKFROMFILE (OLECLI.DEFCREATELINKFROMFILE)
 0000:0000  Imp  DEFLOADFROMSTREAM    (OLECLI.DEFLOADFROMSTREAM)
 0000:0000  Imp  DELETEDC             (GDI.68)
 0000:0000  Imp  DELETEOBJECT         (GDI.69)
 0001:0D40       DLLACTIVATE
 0001:1174       DLLCHANGEDATA
 0001:0AAA       DLLCLONE
 0001:0E9A       DLLCLOSE
 0001:0B52       DLLCOPYFROMLINK
 0001:0BD0       DLLCOPYTOCLIPBOARD
 0001:0678       DllCreate
 0001:0558       DllCreateFromClip
 0001:06DA       DllCreateFromFile
 0001:0616       DllCreateFromTemplate
 0001:05BA       DllCreateLinkFromClip
 0001:0742       DllCreateLinkFromFile
 0001:0A22       DLLDELETE
 0001:0906       DLLDOVERB
 0001:0BF2       DLLDRAW
 0001:09D4       DLLENUMFORMATS
 0001:0BA8       DLLEQUAL
 0001:0E72       DLLEXECUTE
 0001:0932       DLLGETDATA
 0001:0F5C       DLLGETLINKUPDATEOPTIONS
 0001:04F0       DllLoadFromStream
 0001:0F00       DLLOBJECTCONVERT
 0001:1126       DLLOBJECTLONG
 0001:1028       DLLQUERYBOUNDS
 0001:0FD2       DLLQUERYNAME
 0001:1078       DLLQUERYOPEN
 0001:109A       DLLQUERYOUTOFDATE
 0001:0896       DLLQUERYPROTOCOL
 0001:10DE       DLLQUERYRELEASEERROR
 0001:1152       DLLQUERYRELEASEMETHOD
 0001:10BC       DLLQUERYRELEASESTATUS
 0001:1050       DLLQUERYSIZE
 0001:1000       DLLQUERYTYPE
 0001:0EDE       DLLRECONNECT
 0001:08BE       DLLRELEASE
 0001:0FAA       DLLRENAME
 0001:1100       DLLREQUESTDATA
 0001:0A82       DLLSAVETOSTREAM
 0001:09AC       DLLSETBOUNDS
 0001:09FA       DLLSETCOLORSCHEME
 0001:095E       DLLSETDATA
 0001:0A54       DLLSETHOSTNAMES
 0001:0F84       DLLSETLINKUPDATEOPTIONS
 0001:0986       DLLSETTARGETDEVICE
 0001:08E0       DLLSHOW
 0001:0EBC       DLLUPDATE
 0000:0000  Imp  GETACTIVEWINDOW      (USER.60)
 0000:0000  Imp  GETCLIENTRECT        (USER.33)
 0000:0000  Imp  GETCLIPBOX           (GDI.77)
 0000:0000  Imp  GETDCORG             (GDI.79)
 0000:0000  Imp  GETDESKTOPWINDOW     (USER.286)
 0000:0000  Imp  GETFOCUS             (USER.23)
 0000:0000  Imp  GETMODULEFILENAME    (KERNEL.49)
 0001:0CDA       GETOPUSRECT
 0000:0000  Imp  GETWINDOW            (USER.262)
 0000:0000  Imp  GLOBALLOCK           (KERNEL.18)
 0000:0000  Imp  INTERSECTRECT        (USER.79)
 0001:008C       ISAPP
 0000:0000  Imp  ISBADREADPTR         (KERNEL.334)
 0001:00F0       ISDCMEMORY
 0000:0000  Imp  ISRECTEMPTY          (USER.75)
 0000:0000  Imp  ISWINDOW             (USER.47)
 0001:0000       LibEntry
 0001:001C       LibMain
 0000:0000  Imp  LOCALALLOC           (KERNEL.5)
 0000:0000  Imp  LOCALFREE            (KERNEL.7)
 0000:0000  Imp  LocalInit            (KERNEL.4)
 0000:0000  Imp  LPTODP               (GDI.99)
 0000:0000  Imp  LSTRCMPI             (USER.471)
 0000:0000  Imp  LSTRLEN              (KERNEL.90)
 0000:0000  Imp  OFFSETRECT           (USER.77)
 0000:0000  Imp  OLEISDCMETA          (OLECLI.60)
 0001:03DC       OleQueryObjPos
 0000:0000  Imp  OUTPUTDEBUGSTR       (MMSYSTEM.OUTPUTDEBUGSTR)
 0002:0008       pAtomTable
 0002:0006       pLocalHeap
 0002:000E       pStackBot
 0002:000C       pStackMin
 0002:000A       pStackTop
 0000:0000  Imp  PTINRECT             (USER.76)
 0000:0000  Imp  REGSETVALUE          (SHELL.5)
 0002:0006       rsrvptrs
 0000:0000  Imp  SCREENTOCLIENT       (USER.29)
 0000:0000  Imp  SELECTOBJECT         (GDI.45)
 0000:0000  Imp  SETRECTEMPTY         (USER.73)
 0001:0070       WEP
 0001:0860       _CanReplace
 0001:0242       _CleanObjects
 0001:014A       _DelObj
 0001:011C       _FindObj
 0001:0868       _GetData
 0002:00EC       _ghInstance
 0002:018E       _hbmStock
 0001:02E8       _LookForDC
 0002:018A       _lpobjActive
 0001:027E       _NewObj
 0002:0010       _poiFirst
 0001:039C       _RectSameSize
 0001:01A0       _RegSetGetData
 0001:07B0       _ReplaceFunctions
 0002:00EE       _vtblDef
 0002:0050       _vtblDll
 0001:038A       _WindowFromDC
 0000:0000  Imp  _wsprintf            (USER.420)
 0000:0001  Abs  __acrtused

  Address         Publics by Value

 0000:0000  Imp  ISRECTEMPTY          (USER.75)
 0000:0000  Imp  OFFSETRECT           (USER.77)
 0000:0000  Imp  LPTODP               (GDI.99)
 0000:0000  Imp  GETCLIPBOX           (GDI.77)
 0000:0000  Imp  DEFCREATEFROMFILE    (OLECLI.DEFCREATEFROMFILE)
 0000:0000  Imp  DEFCREATEFROMCLIP    (OLECLI.DEFCREATEFROMCLIP)
 0000:0000  Imp  LSTRLEN              (KERNEL.90)
 0000:0000  Imp  GETFOCUS             (USER.23)
 0000:0000  Imp  DELETEOBJECT         (GDI.69)
 0000:0000  Imp  DEFCREATE            (OLECLI.DEFCREATE)
 0000:0000  Imp  GETCLIENTRECT        (USER.33)
 0000:0000  Imp  OLEISDCMETA          (OLECLI.60)
 0000:0000  Imp  LOCALFREE            (KERNEL.7)
 0000:0000  Imp  SELECTOBJECT         (GDI.45)
 0000:0000  Imp  GETDESKTOPWINDOW     (USER.286)
 0000:0000  Imp  ISWINDOW             (USER.47)
 0000:0000  Imp  SETRECTEMPTY         (USER.73)
 0000:0000  Imp  LocalInit            (KERNEL.4)
 0000:0000  Imp  GETACTIVEWINDOW      (USER.60)
 0000:0000  Imp  DEFCREATEFROMTEMPLATE (OLECLI.DEFCREATEFROMTEMPLATE)
 0000:0000  Imp  LSTRCMPI             (USER.471)
 0000:0000  Imp  DEFCREATELINKFROMCLIP (OLECLI.DEFCREATELINKFROMCLIP)
 0000:0000  Imp  DEFCREATELINKFROMFILE (OLECLI.DEFCREATELINKFROMFILE)
 0000:0000  Imp  ISBADREADPTR         (KERNEL.334)
 0000:0000  Imp  SCREENTOCLIENT       (USER.29)
 0000:0000  Imp  PTINRECT             (USER.76)
 0000:0000  Imp  CREATEBITMAP         (GDI.48)
 0000:0000  Imp  OUTPUTDEBUGSTR       (MMSYSTEM.OUTPUTDEBUGSTR)
 0000:0000  Imp  LOCALALLOC           (KERNEL.5)
 0000:0000  Imp  GLOBALLOCK           (KERNEL.18)
 0000:0000  Imp  INTERSECTRECT        (USER.79)
 0000:0000  Imp  CLIENTTOSCREEN       (USER.28)
 0000:0000  Imp  DEFLOADFROMSTREAM    (OLECLI.DEFLOADFROMSTREAM)
 0000:0000  Imp  REGSETVALUE          (SHELL.5)
 0000:0000  Imp  GETMODULEFILENAME    (KERNEL.49)
 0000:0000  Imp  GETWINDOW            (USER.262)
 0000:0000  Imp  CREATECOMPATIBLEDC   (GDI.52)
 0000:0000  Imp  _wsprintf            (USER.420)
 0000:0000  Imp  GETDCORG             (GDI.79)
 0000:0000  Imp  DELETEDC             (GDI.68)
 0000:0001  Abs  __acrtused
 0001:0000       LibEntry
 0001:001C       LibMain
 0001:0070       WEP
 0001:008C       ISAPP
 0001:00F0       ISDCMEMORY
 0001:011C       _FindObj
 0001:014A       _DelObj
 0001:01A0       _RegSetGetData
 0001:0242       _CleanObjects
 0001:027E       _NewObj
 0001:02E8       _LookForDC
 0001:038A       _WindowFromDC
 0001:039C       _RectSameSize
 0001:03DC       OleQueryObjPos
 0001:04F0       DllLoadFromStream
 0001:0558       DllCreateFromClip
 0001:05BA       DllCreateLinkFromClip
 0001:0616       DllCreateFromTemplate
 0001:0678       DllCreate
 0001:06DA       DllCreateFromFile
 0001:0742       DllCreateLinkFromFile
 0001:07B0       _ReplaceFunctions
 0001:0860       _CanReplace
 0001:0868       _GetData
 0001:0896       DLLQUERYPROTOCOL
 0001:08BE       DLLRELEASE
 0001:08E0       DLLSHOW
 0001:0906       DLLDOVERB
 0001:0932       DLLGETDATA
 0001:095E       DLLSETDATA
 0001:0986       DLLSETTARGETDEVICE
 0001:09AC       DLLSETBOUNDS
 0001:09D4       DLLENUMFORMATS
 0001:09FA       DLLSETCOLORSCHEME
 0001:0A22       DLLDELETE
 0001:0A54       DLLSETHOSTNAMES
 0001:0A82       DLLSAVETOSTREAM
 0001:0AAA       DLLCLONE
 0001:0B52       DLLCOPYFROMLINK
 0001:0BA8       DLLEQUAL
 0001:0BD0       DLLCOPYTOCLIPBOARD
 0001:0BF2       DLLDRAW
 0001:0CDA       GETOPUSRECT
 0001:0D40       DLLACTIVATE
 0001:0E72       DLLEXECUTE
 0001:0E9A       DLLCLOSE
 0001:0EBC       DLLUPDATE
 0001:0EDE       DLLRECONNECT
 0001:0F00       DLLOBJECTCONVERT
 0001:0F5C       DLLGETLINKUPDATEOPTIONS
 0001:0F84       DLLSETLINKUPDATEOPTIONS
 0001:0FAA       DLLRENAME
 0001:0FD2       DLLQUERYNAME
 0001:1000       DLLQUERYTYPE
 0001:1028       DLLQUERYBOUNDS
 0001:1050       DLLQUERYSIZE
 0001:1078       DLLQUERYOPEN
 0001:109A       DLLQUERYOUTOFDATE
 0001:10BC       DLLQUERYRELEASESTATUS
 0001:10DE       DLLQUERYRELEASEERROR
 0001:1100       DLLREQUESTDATA
 0001:1126       DLLOBJECTLONG
 0001:1152       DLLQUERYRELEASEMETHOD
 0001:1174       DLLCHANGEDATA
 0002:0006       rsrvptrs
 0002:0006       pLocalHeap
 0002:0008       pAtomTable
 0002:000A       pStackTop
 0002:000C       pStackMin
 0002:000E       pStackBot
 0002:0010       _poiFirst
 0002:0050       _vtblDll
 0002:00EC       _ghInstance
 0002:00EE       _vtblDef
 0002:018A       _lpobjActive
 0002:018E       _hbmStock

Program entry point at 0001:0000
